:020000020000FC
:10000000FFC062C579C579C579C579C5B1C5A6C531
:10001000A6C5A6C5A2C58EC58EC58EC588C588C510
:1000200088C5A7C59EC59EC59EC5A4C5A0C59EC5BD
:04003000A2C5A2C5FE
:10020000F89400E810E0009361001093610000E3AF
:1002100005B90FEF04B900E008B90FED07B906E41E
:100220000BB909EF0AB9B1E0A0E0D3E0C0E000E00B
:100230000D93BD17E9F7AC17D9F712E00EEF1EBF0B
:100240000DBF00E005BF03E00CBB00E105BB01E210
:1002500004BD0BE005BD00E006BD02E307BD00E004
:1002600008BD00E003BD00E00093800003E00093C0
:10027000810000E00093820010E000E01093850010
:100280000093840010E000E0109389000093880040
:1002900010E000E010938B0000938A0010E000E073
:1002A000109387000093860000E107BB01E20093F2
:1002B000B0000CE00093B10000E00093B20002E354
:1002C0000093B30000E00093B40000E00093B60098
:1002D00007EE00937C0005EE00937A0000E00093A7
:1002E0007B0000E000937E0000E80093300000E017
:1002F00000937F0010E003E01093C5000093C4005A
:1003000002E20093C00000E00093C10006E0009309
:10031000C20000E000937B0001E000936900A89513
:1003200008E1009360000EE00093600002E8009393
:10033000640001E00DBB04E00093680000E000935E
:100340006B0000E000936C0002E000936D0000E0A1
:1003500000936E0001E000936F0000E000937000D6
:100360000AE0202E0AE0402E04E60093100106E980
:100370000093110106E90093120108EC00931301A8
:1003800004E6009330010DE7009331010CE800937F
:10039000320108EC009333010CE80093500102E0B5
:1003A0000093510108E2009355010091120100935E
:1003B0001A0100931B010091320100933A0100934E
:1003C0003B010AE00093600190E081E149D40F3FD6
:1003D000D1F00093110182E143D40093120180E334
:1003E0003FD40093300181E33BD40093310182E399
:1003F00037D40093320183E333D40093330181E592
:100400002FD400935101789406E9A89591FFFDCF70
:100410009D7F0A95D1F704B700FF0EC00E7F04BF81
:100420001AEFA89591FFFDCF9D7F1A9509F461C23F
:1004300000913A01043BA8F7009133011091320179
:10044000011B009336010091320110913001011B14
:10045000009334010091320110913101011B08F425
:1004600000E0009335010091130110911201011B6E
:10047000009316010091120110911001011B0093CD
:10048000140110915101113011F40EE70AC012301D
:1004900011F400EA06C0133011F400EF02C000EFBF
:1004A00000C000935201309151015E980AEFE2D3EF
:1004B0005E9A0AEFDFD30AEFDDD33A95B1F70AEF80
:1004C000D9D30AEFD7D30AEFD5D35E98A89591FF79
:1004D0000FC29D7F5E9893FD17C01091320120914D
:1004E000320135E0131B230F00913A015ED320F453
:1004F0000AE000936001FCC1009160010A9500933D
:10050000600109F0F5C1986002E0402E9F7E0091E5
:100510001A0110911B01011B99F008F408C023E097
:10052000033008F421E0120F10931B0109C001955C
:1005300023E0033008F421E0121B10931B0100C0DC
:1005400000913A0110913B01011B99F008F408C099
:1005500023E0033008F421E0120F10933B0109C09F
:10056000019523E0033008F421E0121B10933B01B6
:1005700000C092FD17C000917800009179001091A1
:100580005201011720F008E20093550122C00091AA
:1005900055010A950093550121F408E20093550195
:1005A000946017C000917800009179001091520179
:1005B000011720F408E2009355010BC0009155018A
:1005C0000A950093550121F408E2009355019B7FA1
:1005D00000C092FF01C088C100911B01109112015F
:1005E000011B00931C0100913B0110913201011B82
:1005F00000933C0100913C0107FD71C0055008F4D7
:10060000FEC09F7D05B105FD02C00FEF33D32C9ACC
:100610002D9A0091360107BD0093B30000911C0193
:1006200007FF15C000911C01019510913C0120911C
:100630001601FBD210913C01010F10911301209182
:100640001101121B20911601F0D2DDD217C00091CA
:100650001C0110913C0120911601E7D2102F00914E
:100660003C01011B08F400E01091130120911101DD
:10067000121B20911601D9D2C6D200C000911C01D4
:1006800007FF18C000911C01019510913C012091B9
:100690001401CBD2102F00913C01011B08F400E0A3
:1006A0002091100110911101121B20911401BDD253
:1006B000B2D214C000911C0110913C012091140190
:1006C000B4D210913C01010F209110011091110141
:1006D000121B20911401A9D29ED200C009C1009121
:1006E0003C010195055008F48AC09F7D05B105FFC6
:1006F00002C00FEFBFD22C982D980091340107BD96
:100700000093B30000911C0107FF1CC000911C0165
:10071000019510913C0111952091160186D21091FE
:100720003C011195010F10913501209134017DD2CA
:100730001091130120911101121B2091160175D205
:1007400062D21EC000911C0110913C0111952091B4
:1007500016016BD210913C011195101B08F410E0AA
:10076000012F10913501209134015FD210911301B6
:1007700020911101121B2091160157D244D200C0C2
:1007800000911C0107FF1FC000911C0101951091F1
:100790003C0111952091140148D210913C01119512
:1007A000101B08F410E0012F109135012091340145
:1007B0003CD22091100110911101121B20911401C3
:1007C00034D229D21BC000911C0110913C0111951B
:1007D000209114012AD210913C011195010F109122
:1007E00035012091340121D2209110011091110185
:1007F000121B2091140119D20ED200C079C01091A1
:1008000012012091120135E0131B230F00911B01EF
:10081000CCD108F401C0906295FF66C0109112011E
:100820002091120135E0131B230F00911B01BDD154
:1008300008F05AC000911C0107FD2AC005B105FD52
:1008400002C00FEF17D22C982D9A10911601109319
:10085000B30000911C012091100110911101121B95
:1008600020911401E2D1D7D11091160117BD00914A
:100870001C011091350120913401D7D11091130141
:1008800020911101121B20911601CFD1BCD130C093
:1008900005B105FF02C00FEFEDD12C9A2D981091F4
:1008A000140117BD00911C010195109113012091B5
:1008B0001101121B20911601B8D1A5D1109114017C
:1008C0001093B30000911C01019510913501209106
:1008D0003401ABD12091100110911101121B209114
:1008E0001401A3D198D104C000E008BD0093B40066
:1008F000EDCD11E004E6BED11A95E1F714EB2CED35
:1009000000913A010093330150D108F4D6C012E8A7
:100910002AEA00911A010093120147D108F4CDC0D0
:1009200075EA5E980AEFA6D15E9A12E304E6A2D1B8
:100930001A95E1F710E522E800913A0100933001A1
:1009400034D108F4BAC05E980AEF94D15E9A12E3EB
:1009500004E690D11A95E1F7109130012AE0120FC8
:1009600020EA00913A01009332011FD108F4A5C09A
:100970005E980AEF7FD15E9A12E304E67BD11A9566
:10098000E1F710913001209132013AE0230F0091FC
:100990003A010093310109D108F48FC05E980AEF43
:1009A00069D15E9A12E304E665D11A95E1F70091E8
:1009B0003A01009350013AE0109133012091330144
:1009C000131B230F00915001F0D020F003E000939F
:1009D000510124C0109132012091320135E0131BE6
:1009E0003AE0230F00915001E0D020F002E00093A4
:1009F000510114C010913001209130013AE0131BD5
:100A000035E0230F00915001D0D020F001E0009399
:100A1000510104C002E0009351014FC05E980AEFFB
:100A200029D15E9A12E304E625D11A95E1F70091E7
:100A30001A01009311013AE0109133012091330122
:100A4000131B230F00913A01B0D008F436C0009177
:100A5000110181E1F6D00091120182E1F2D0009102
:100A6000300180E3EED00091310181E3EAD00091C2
:100A7000320182E3E6D00091330183E3E2D00091BA
:100A8000510181E5DED070E0309151015E980AEFAE
:100A9000F1D05E9A0AEFEED00AEFECD03A95B1F7BA
:100AA0000AEFE8D00AEFE6D00AEFE4D00AEFE2D08E
:100AB0000AEFE0D00AEFDED0E7CF5E9806E4DAD0A6
:100AC0005E9A06E4D7D0F9CFFFB60F931F9300913B
:100AD00084004A9903C0009318010AC000931901C9
:100AE00010911801011B023318F000931A01916054
:100AF0001F910F91FFBE1895189518951895FFB680
:100B00000F931F9300918400499903C0009338010B
:100B10000AC00093390110913801011B023318F00B
:100B200000933A0192601F910F91FFBE189518959E
:100B30001895189518951895FFB64A9461F4906128
:100B40000F935E9A00911A0100931B0100E008BD0B
:100B50000093B4000F91FFBE18951895189518953D
:100B6000189518951895189518951895189518951D
:100B70001895189518951895189510E010937A0007
:100B800010917C00107F102B10937C0000E00093EC
:100B90007B0005EC00937A0000917A0006FDFCCF03
:100BA00000917800109179000895011710F0201736
:100BB00000F008956F937F93712F602F621B730B6A
:100BC00028F0712F602F461B570B00F07F916F911B
:100BD00008954F935F936F934427552760E1000F6B
:100BE000111F441F551F4217530718F00395421B4E
:100BF000530B6A95A1F75F934F932F913F916F919C
:100C00005F914F9108951F9317B5011708F0012FB9
:100C100008BD1F9108951F931091B300011708F0AC
:100C2000012F0093B4001F9108950F921F923F93DC
:100C3000019F112D002D30E0CCDF3F911F900F90D0
:100C400008951F93F999FECF10E01FBB10E012BD6D
:100C500081BD00BD753A11F4FA9AF99A1F91089571
:100C60001F93F999FECF10E012BD81BDF89A00B52F
:100C70001F9108951F932F93A89519E02DEE2A95A3
:100C8000F1F71A95D9F70A95B9F72F911F910895A1
:00000001FF
